 sgx_init_test

 Timestamp is 4be8c2cf (Tue May 11 11:37:03 2010)

 Preferred load address is 00010000

 Start         Length     Name                   Class
 0001:00000000 00000004H .CRT$XCA                CODE
 0001:00000004 00000004H .CRT$XCZ                CODE
 0001:00000008 00000004H .CRT$XIA                CODE
 0001:0000000c 00000004H .CRT$XIZ                CODE
 0001:00000010 00000004H .CRT$XPA                CODE
 0001:00000014 00000004H .CRT$XPZ                CODE
 0001:00000018 00000004H .CRT$XTA                CODE
 0001:0000001c 00000004H .CRT$XTZ                CODE
 0001:00000020 00001080H .rdata                  CODE
 0001:000010a0 0000002aH .rdata$debug            CODE
 0001:000010cc 000018d4H .text                   CODE
 0001:000029a0 0000001cH .xdata                  CODE
 0001:000029bc 00000028H .idata$2                CODE
 0001:000029e4 00000014H .idata$3                CODE
 0001:000029f8 000000a4H .idata$4                CODE
 0001:00002a9c 000000eaH .idata$6                CODE
 0001:00002b86 00000000H .edata                  CODE
 0002:00000000 000000a4H .idata$5                DATA
 0002:000000a4 00000008H .data                   DATA
 0002:000000ac 00000010H .bss                    DATA
 0003:00000000 00000088H .pdata                  DATA

  Address         Publics by Value              Rva+Base       Lib:Object

 0000:00000000       ___safe_se_handler_count   00000000     <absolute>
 0000:00000000       ___safe_se_handler_table   00000000     <absolute>
 0001:00000000       __xc_a                     00011000     corelib0:crt0init.obj
 0001:00000004       __xc_z                     00011004     corelib0:crt0init.obj
 0001:00000008       __xi_a                     00011008     corelib0:crt0init.obj
 0001:0000000c       __xi_z                     0001100c     corelib0:crt0init.obj
 0001:00000010       __xp_a                     00011010     corelib0:crt0init.obj
 0001:00000014       __xp_z                     00011014     corelib0:crt0init.obj
 0001:00000018       __xt_a                     00011018     corelib0:crt0init.obj
 0001:0000001c       __xt_z                     0001101c     corelib0:crt0init.obj
 0001:0000003c       ??_C@_0BD@FOHFKAOE@INVALID?5ERROR?5CODE?$AA@ 0001103c     sgx_init_test.obj
 0001:00000050       ??_C@_09KMCHPOPM@PVRSRV_OK?$AA@ 00011050     sgx_init_test.obj
 0001:0000005c       ??_C@_0BF@KHEAJDEG@PVRSRV_ERROR_GENERIC?$AA@ 0001105c     sgx_init_test.obj
 0001:00000074       ??_C@_0BL@BOENCAIM@PVRSRV_ERROR_OUT_OF_MEMORY?$AA@ 00011074     sgx_init_test.obj
 0001:00000090       ??_C@_0BN@IHBDMIPO@PVRSRV_ERROR_TOO_FEW_BUFFERS?$AA@ 00011090     sgx_init_test.obj
 0001:000000b0       ??_C@_0BO@EGNEIFEA@PVRSRV_ERROR_SYMBOL_NOT_FOUND?$AA@ 000110b0     sgx_init_test.obj
 0001:000000d0       ??_C@_0BL@BKMGFOLH@PVRSRV_ERROR_OUT_OF_HSPACE?$AA@ 000110d0     sgx_init_test.obj
 0001:000000ec       ??_C@_0BM@LGNAOM@PVRSRV_ERROR_INVALID_PARAMS?$AA@ 000110ec     sgx_init_test.obj
 0001:00000108       ??_C@_0BN@MGJEIKFE@PVRSRV_ERROR_TILE_MAP_FAILED?$AA@ 00011108     sgx_init_test.obj
 0001:00000128       ??_C@_0BK@JHPIKHJG@PVRSRV_ERROR_INIT_FAILURE?$AA@ 00011128     sgx_init_test.obj
 0001:00000144       ??_C@_0CE@POPMCOCG@PVRSRV_ERROR_CANT_REGISTER_CALLB@ 00011144     sgx_init_test.obj
 0001:00000168       ??_C@_0BM@COIEDMNF@PVRSRV_ERROR_INVALID_DEVICE?$AA@ 00011168     sgx_init_test.obj
 0001:00000184       ??_C@_0BH@OEOFFCIM@PVRSRV_ERROR_NOT_OWNER?$AA@ 00011184     sgx_init_test.obj
 0001:0000019c       ??_C@_0BJ@PHFCJIBD@PVRSRV_ERROR_BAD_MAPPING?$AA@ 0001119c     sgx_init_test.obj
 0001:000001b8       ??_C@_0BF@KGIMOMJE@PVRSRV_ERROR_TIMEOUT?$AA@ 000111b8     sgx_init_test.obj
 0001:000001d0       ??_C@_0BI@CDPBDDFH@PVRSRV_ERROR_NO_PRIMARY?$AA@ 000111d0     sgx_init_test.obj
 0001:000001e8       ??_C@_0BP@FMELGOJO@PVRSRV_ERROR_FLIP_CHAIN_EXISTS?$AA@ 000111e8     sgx_init_test.obj
 0001:00000208       ??_C@_0BN@JMHJCLJP@ERROR_CANNOT_ACQUIRE_SYSDATA?$AA@ 00011208     sgx_init_test.obj
 0001:00000228       ??_C@_0BL@JPEIBKNH@PVRSRV_ERROR_SCENE_INVALID?$AA@ 00011228     sgx_init_test.obj
 0001:00000244       ??_C@_0BK@JAAFMMBM@PVRSRV_ERROR_STREAM_ERROR?$AA@ 00011244     sgx_init_test.obj
 0001:00000260       ??_C@_0DP@FHJOPEMA@PVRSRV_ERROR_INVALID_INTERRUPTPV@ 00011260     sgx_init_test.obj
 0001:000002a0       ??_C@_0BP@PFBLKCEO@PVRSRV_ERROR_CMD_NOT_PROCESSED?$AA@ 000112a0     sgx_init_test.obj
 0001:000002c0       ??_C@_0BJ@PHLIKBPN@PVRSRV_ERROR_CMD_TOO_BIG?$AA@ 000112c0     sgx_init_test.obj
 0001:000002dc       ??_C@_0CE@FHHHLEGE@PVRSRV_ERROR_DEVICE_REGISTER_FAI@ 000112dc     sgx_init_test.obj
 0001:00000300       ??_C@_0BI@JBKNPCOM@PVRSRV_ERROR_FIFO_SPACE?$AA@ 00011300     sgx_init_test.obj
 0001:00000318       ??_C@_0BJ@IIGHNIEG@PVRSRV_ERROR_TA_RECOVERY?$AA@ 00011318     sgx_init_test.obj
 0001:00000334       ??_C@_0BN@BKNBJNB@PVRSRV_ERROR_INDOSORLOWPOWER?$AA@ 00011334     sgx_init_test.obj
 0001:00000354       ??_C@_0BM@MCHBLHIP@PVRSRV_ERROR_TOOMANYBUFFERS?$AA@ 00011354     sgx_init_test.obj
 0001:00000370       ??_C@_0BL@FINKNLDE@PVRSRV_ERROR_NOT_SUPPORTED?$AA@ 00011370     sgx_init_test.obj
 0001:0000038c       ??_C@_0CA@KIDKOOGL@PVRSRV_ERROR_PROCESSING_BLOCKED?$AA@ 0001138c     sgx_init_test.obj
 0001:000003ac       ??_C@_0CA@NBGAMPKE@PVRSRV_ERROR_CANNOT_FLUSH_QUEUE?$AA@ 000113ac     sgx_init_test.obj
 0001:000003cc       ??_C@_0CE@NLLBGAEA@PVRSRV_ERROR_CANNOT_GET_QUEUE_SP@ 000113cc     sgx_init_test.obj
 0001:000003f0       ??_C@_0CG@FCILKACH@PVRSRV_ERROR_CANNOT_GET_RENDERDE@ 000113f0     sgx_init_test.obj
 0001:00000418       ??_C@_0BD@COEEPPOL@PVRSRV_ERROR_RETRY?$AA@ 00011418     sgx_init_test.obj
 0001:0000042c       ??_C@_0BJ@IMBALOKG@PVRSRV_DEVICE_ID_UNKNOWN?$AA@ 0001142c     sgx_init_test.obj
 0001:00000448       ??_C@_0BH@OGEGGGCD@PVRSRV_DEVICE_ID_MSVDX?$AA@ 00011448     sgx_init_test.obj
 0001:00000460       ??_C@_0BF@BBCLGMON@PVRSRV_DEVICE_ID_SGX?$AA@ 00011460     sgx_init_test.obj
 0001:00000478       ??_C@_0CD@BDGFMHBG@PVRSRV_DEVICE_TYPE_EXT?5?$CI3rd?5Part@ 00011478     sgx_init_test.obj
 0001:0000049c       ??_C@_0BE@GEDKFGMC@Not?5recognised?50x?$CFx?$AA@ 0001149c     sgx_init_test.obj
 0001:000004b0       ??_C@_0BI@ICLDLMDM@?4?4?4?4?5ui32ProcessID?3?$CFlu?6?$AA@ 000114b0     sgx_init_test.obj
 0001:000004c8       ??_C@_09JLJAGNAE@disabled?6?$AA@ 000114c8     sgx_init_test.obj
 0001:000004d4       ??_C@_08EHJFGCDI@enabled?6?$AA@ 000114d4     sgx_init_test.obj
 0001:000004e0       ??_C@_0CD@PBGAODGL@?4?4?4?4?5USE_SUPPORT_NO_TA3D_OVERLAP@ 000114e0     sgx_init_test.obj
 0001:00000504       ??_C@_0CH@KDLNALHG@?4?4?4?4?5SUPPORT_SGX_PRIORITY_SCHEDU@ 00011504     sgx_init_test.obj
 0001:0000052c       ??_C@_0CC@PBEBICKP@?4?4?4?4?5SUPPORT_SGX_MMU_DUMMY_PAGE?3@ 0001152c     sgx_init_test.obj
 0001:00000550       ??_C@_0BK@JEEICFNJ@?4?4?4?4?5SUPPORT_SGX_HWPERF?3?5?$AA@ 00011550     sgx_init_test.obj
 0001:0000056c       ??_C@_0BN@IKKPFPFH@?4?4?4?4?5SUPPORT_PERCONTEXT_PB?3?5?$AA@ 0001156c     sgx_init_test.obj
 0001:0000058c       ??_C@_0CI@KGPIAJLH@?4?4?4?4?5SUPPORT_DISPLAYCONTROLLER_T@ 0001158c     sgx_init_test.obj
 0001:000005b4       ??_C@_0CH@FMAMMJDI@?4?4?4?4?5SUPPORT_ACTIVE_POWER_MANAGE@ 000115b4     sgx_init_test.obj
 0001:000005dc       ??_C@_0BP@EKNECPM@?4?4?4?4?5SGX_SUPPORT_HWPROFILING?3?5?$AA@ 000115dc     sgx_init_test.obj
 0001:000005fc       ??_C@_0CA@EGNBMLMJ@?4?4?4?4?5SGX_FEATURE_SYSTEM_CACHE?3?5?$AA@ 000115fc     sgx_init_test.obj
 0001:0000061c       ??_C@_0CI@JFPPAJCE@?4?4?4?4?5SGX_FEATURE_RENDER_TARGET_A@ 0001161c     sgx_init_test.obj
 0001:00000644       ??_C@_0CC@NPOADBLC@?4?4?4?4?5SGX_FEATURE_OVERLAPPED_SPM?3@ 00011644     sgx_init_test.obj
 0001:00000668       ??_C@_0CB@ODIPCGL@?4?4?4?4?5SGX_FEATURE_MP_CORE_COUNT?3?5@ 00011668     sgx_init_test.obj
 0001:0000068c       ??_C@_04PEDNGLFL@?$CFld?6?$AA@ 0001168c     sgx_init_test.obj
 0001:00000694       ??_C@_0CJ@CGFGFCIK@?4?4?4?4?5SGX_FEATURE_MULTITHREADED_U@ 00011694     sgx_init_test.obj
 0001:000006c0       ??_C@_0BG@EHGIBNPN@?4?4?4?4?5SGX_FEATURE_MP?3?5?$AA@ 000116c0     sgx_init_test.obj
 0001:000006d8       ??_C@_0BH@CEHELPHH@?4?4?4?4?5SGX_FEATURE_DCU?3?5?$AA@ 000116d8     sgx_init_test.obj
 0001:000006f0       ??_C@_0BJ@NDCCFHBD@?4?4?4?4?5SGX_FAST_DPM_INIT?3?5?$AA@ 000116f0     sgx_init_test.obj
 0001:0000070c       ??_C@_0CE@LFDOJJDJ@?4?4?4?4?5SGX_DONT_SWITCH_OFF_FEATURE@ 0001170c     sgx_init_test.obj
 0001:00000730       ??_C@_0BK@DFJDHFPM@?4?4?4?4?5SGX_DMS_AGE_ENABLE?3?5?$AA@ 00011730     sgx_init_test.obj
 0001:0000074c       ??_C@_0BP@CMJHKMAD@?4?4?4?4?5SGX_BYPASS_SYSTEM_CACHE?3?5?$AA@ 0001174c     sgx_init_test.obj
 0001:0000076c       ??_C@_0BK@EFNNGEBJ@?4?4?4?4?5PVR_SECURE_HANDLES?3?5?$AA@ 0001176c     sgx_init_test.obj
 0001:00000788       ??_C@_0BL@MHAEDBH@?4?4?4?4?5SUPPORT_HW_RECOVERY?3?5?$AA@ 00011788     sgx_init_test.obj
 0001:000007a4       ??_C@_0CE@EBOHCEFA@?4?4?4?4?5PVRSRV_USSE_EDM_STATUS_DEBU@ 000117a4     sgx_init_test.obj
 0001:000007c8       ??_C@_0N@CBKLAPJJ@?4?4?4?4?5PDUMP?3?5?$AA@ 000117c8     sgx_init_test.obj
 0001:000007d8       ??_C@_0DA@JOODEMOL@?4?4?4?4?5SGX?5microkernel?5DDK?5version@ 000117d8     sgx_init_test.obj
 0001:00000808       ??_C@_0DP@OBEHLMF@?4?4?4?4?5SGX?5microkernel?5software?5co@ 00011808     sgx_init_test.obj
 0001:00000848       ??_C@_0BP@GFIFMEMA@SGX?5microkernel?5build?5options?6?$AA@ 00011848     sgx_init_test.obj
 0001:00000868       ??_C@_0N@PMKALKLK@?4?4?4?4?5DEBUG?3?5?$AA@ 00011868     sgx_init_test.obj
 0001:00000878       ??_C@_0BM@LFGEPCCF@?4?4?4?4?5Hardware?5core?5ID?3?5?$CFld?6?$AA@ 00011878     sgx_init_test.obj
 0001:00000894       ??_C@_0CG@PMKABEN@?4?4?4?4?5Hardware?5core?5ID?3?5?$CFld?0?5name@ 00011894     sgx_init_test.obj
 0001:000008ba       ??_C@_00CNPNBAHC@?$AA@     000118ba     sgx_init_test.obj
 0001:000008bc       ??_C@_0M@JDCKMKKM@SGX?5520?1530?$AA@ 000118bc     sgx_init_test.obj
 0001:000008c8       ??_C@_07KCCNKLDG@SGX?5535?$AA@ 000118c8     sgx_init_test.obj
 0001:000008d0       ??_C@_07NKBFEJPG@SGX?5540?$AA@ 000118d0     sgx_init_test.obj
 0001:000008d8       ??_C@_07KHGCLNLD@SGX?5545?$AA@ 000118d8     sgx_init_test.obj
 0001:000008e0       ??_C@_07MGEBGODC@SGX?5531?$AA@ 000118e0     sgx_init_test.obj
 0001:000008e8       ??_C@_0L@FANDILD@SGX?554x?9MP?$AA@ 000118e8     sgx_init_test.obj
 0001:000008f4       ??_C@_0DN@PDOMMKDJ@?4?4?4?4?5Hardware?5core?5designer?3?5?$CFd?0@ 000118f4     sgx_init_test.obj
 0001:00000934       ??_C@_0DA@FHGIJGL@?4?4?4?4?5SGX?5Host?5driver?5DDK?5version@ 00011934     sgx_init_test.obj
 0001:00000964       ??_C@_0DI@JECPMKED@Misc?5Info?5API?3?5Query?5the?5SGX?5fea@ 00011964     sgx_init_test.obj
 0001:0000099c       ??_C@_04LNELOFCG@?5OK?6?$AA@ 0001199c     sgx_init_test.obj
 0001:000009a4       ??_C@_0M@FBGHFOFL@?5FAIL?5?9?5?$CFs?6?$AA@ 000119a4     sgx_init_test.obj
 0001:000009b0       ??_C@_0DI@JAJOLEGH@Misc?5Info?5API?3?5Query?5the?5SGX?5fea@ 000119b0     sgx_init_test.obj
 0001:000009e8       ??_C@_06HEMPAKAM@?5FAIL?6?$AA@ 000119e8     sgx_init_test.obj
 0001:000009f0       ??_C@_0DH@PINPAELL@?9?9?9?9?9?9?9?9?9?9?9?9?9?9?9?9?9?9?9?9?9End?5loop?5?$CFd@ 000119f0     sgx_init_test.obj
 0001:00000a28       ??_C@_0BD@NOILHFAN@PVRSRVDisconnect?3?6?$AA@ 00011a28     sgx_init_test.obj
 0001:00000a3c       ??_C@_0BH@LMCBNGLN@SGXReleaseClientInfo?3?6?$AA@ 00011a3c     sgx_init_test.obj
 0001:00000a54       ??_C@_0CF@DBFHMBAF@Display?5Class?5API?3?5close?5the?5dev@ 00011a54     sgx_init_test.obj
 0001:00000a7c       ??_C@_0CM@LDEJMMMA@Attempt?5to?5destroy?5memory?5contex@ 00011a7c     sgx_init_test.obj
 0001:00000aa8       ??_C@_0DD@GODBIEMM@Display?5Class?5API?3?5unmap?5display@ 00011aa8     sgx_init_test.obj
 0001:00000adc       ??_C@_0CP@IFAFGPME@Display?5Class?5API?3?5map?5display?5s@ 00011adc     sgx_init_test.obj
 0001:00000b10       ??_C@_0EK@BPNJOJAB@?4?4?4?4?5Shared?5heap?5?$CFlu?5?9?5HeapID?30x@ 00011b10     sgx_init_test.obj
 0001:00000b5c       ??_C@_0DE@BODOPOHG@Display?5Class?5API?3?5get?5the?5syste@ 00011b5c     sgx_init_test.obj
 0001:00000b90       ??_C@_0ED@NNKEOJPF@?4?4?4?4?5Display?5dimensions?5?$CFlu?5?9?5By@ 00011b90     sgx_init_test.obj
 0001:00000bd4       ??_C@_0DB@DPDHNDGF@Display?5Class?5API?3?5enumerate?5dis@ 00011bd4     sgx_init_test.obj
 0001:00000c08       ??_C@_0CK@PAKBMFJN@?4?4?4?4?5Display?5format?5?$CFlu?5?9?5Pixelf@ 00011c08     sgx_init_test.obj
 0001:00000c34       ??_C@_0O@GDPIEJBG@?4?4?4?4?5Name?3?$CFs?6?$AA@ 00011c34     sgx_init_test.obj
 0001:00000c44       ??_C@_0BI@BLGHILNJ@?4?4?4?4?5MaxSwapChains?3?$CFlu?6?$AA@ 00011c44     sgx_init_test.obj
 0001:00000c5c       ??_C@_0BO@POAFDAJE@?4?4?4?4?5MaxSwapChainBuffers?3?$CFlu?6?$AA@ 00011c5c     sgx_init_test.obj
 0001:00000c7c       ??_C@_0BK@CPCAOBID@?4?4?4?4?5MinSwapInterval?3?$CFlu?6?$AA@ 00011c7c     sgx_init_test.obj
 0001:00000c98       ??_C@_0BK@DMGFAHCI@?4?4?4?4?5MaxSwapInterval?3?$CFlu?6?$AA@ 00011c98     sgx_init_test.obj
 0001:00000cb4       ??_C@_0CO@GIPBIACE@Display?5Class?5API?3?5enumerate?5dis@ 00011cb4     sgx_init_test.obj
 0001:00000ce4       ??_C@_0CF@FMDFFMKC@Display?5Class?5API?3?5Get?5display?5i@ 00011ce4     sgx_init_test.obj
 0001:00000d0c       ??_C@_0CA@DAONOMAK@Display?5Class?5API?3?5open?5device?6?$AA@ 00011d0c     sgx_init_test.obj
 0001:00000d2c       ??_C@_0CL@DNLHEBLI@Attempt?5to?5create?5memory?5context@ 00011d2c     sgx_init_test.obj
 0001:00000d58       ??_C@_0CA@DGGJNKGO@?5Test?5Memory?5Allocation?5FAILED?6?$AA@ 00011d58     sgx_init_test.obj
 0001:00000d78       ??_C@_0DM@CIPNLPOO@PVRSRVEnumerateDeviceClass?$CI?$CJ?5ret@ 00011d78     sgx_init_test.obj
 0001:00000db4       ??_C@_0CG@MMBLEMBO@Display?5Class?5API?3?5enumerate?5dev@ 00011db4     sgx_init_test.obj
 0001:00000ddc       ??_C@_0BJ@NLALCGOE@Getting?5SGX?5Client?5info?6?$AA@ 00011ddc     sgx_init_test.obj
 0001:00000df8       ??_C@_0BP@IDIGABKI@Attempt?5to?5acquire?5device?5?$CFd?3?6?$AA@ 00011df8     sgx_init_test.obj
 0001:00000e18       ??_C@_0BH@PPGIPGOP@?5?5?5?5?5?5?5?5?5?5?5?5?$CF04d?5?5?5?5?$HM?5?$AA@ 00011e18     sgx_init_test.obj
 0001:00000e30       ??_C@_01EEMJAFIK@?6?$AA@   00011e30     sgx_init_test.obj
 0001:00000e34       ??_C@_0BK@GEDDINJE@?4?4?4?4?5Reported?5?$CFu?5devices?6?$AA@ 00011e34     sgx_init_test.obj
 0001:00000e50       ??_C@_0CD@INKLJIDI@?4?4?4?4?5Device?5Number?5?5?$HM?5Device?5Typ@ 00011e50     sgx_init_test.obj
 0001:00000e74       ??_C@_0DE@KAFOOJDI@Get?5number?5of?5devices?5from?5PVRSR@ 00011e74     sgx_init_test.obj
 0001:00000ea8       ??_C@_0EA@LNIAFGAD@Try?5calling?5PVRSRVEnumerateDevic@ 00011ea8     sgx_init_test.obj
 0001:00000ee8       ??_C@_0CL@KFFMIBHA@Call?5PVRSRVConnect?5with?5a?5valid?5@ 00011ee8     sgx_init_test.obj
 0001:00000f14       ??_C@_0DH@PPPHAACG@?9?9?9?9?9?9?9?9?9?9?9?9?9?9?9?9?9?9?9?9?9?9?9?5Start?5?9?9@ 00011f14     sgx_init_test.obj
 0001:00000f4c       ??_C@_0DF@NBHKCIFP@Try?5calling?5PVRSRVConnect?5with?5a@ 00011f4c     sgx_init_test.obj
 0001:00000f88       ??_C@_1KE@BDGMONOJ@?$AAH?$AA?3?$AA?2?$AAW?$AAI?$AAN?$AAC?$AAE?$AA6?$AA0?$AA0?$AA?2?$AAP?$AAL?$AAA?$AAT?$AAF?$AAO?$AAR?$AAM?$AA?2?$AAS?$AAM?$AAD?$AAK?$AAV?$AA2?$AA1?$AA0?$AA?2?$AAS?$AAR@ 00011f88     wince_unittests.obj
 0001:0000102c       ??_C@_1CI@OHCJFJPM@?$AAE?$AAR?$AAR?$AAO?$AAR?$AA?3?$AA?5?$AA?$CF?$AAs?$AA?5?$AAl?$AAi?$AAn?$AAe?$AA?5?$AA?$CF?$AAd?$AA?3?$AA?5?$AA?$AA@ 0001202c     wince_unittests.obj
 0001:00001054       ??_C@_1CK@MPGKAOE@?$AA?$CI?$AAe?$AAr?$AAr?$AAo?$AAr?$AA?5?$AAc?$AAo?$AAd?$AAe?$AA?3?$AA?5?$AA?$CF?$AAd?$AA?$CJ?$AA?3?$AA?5?$AA?$CF?$AAs?$AA?$AA@ 00012054     wince_unittests.obj
 0001:00001080       ??_C@_1M@DMCDIEDK@?$AAP?$AAK?$AAM?$AA1?$AA?3?$AA?$AA@ 00012080     wince_unittests.obj
 0001:0000108c       ??_C@_0L@GPAGIAIC@?9disablepm?$AA@ 0001208c     wince_unittests.obj
 0001:00001098       ??_C@_07FBLHGNAH@app?4exe?$AA@ 00012098     wince_unittests.obj
 0001:00001288       print_dev_type             00012288 f   sgx_init_test.obj
 0001:00001870       main                       00012870 f   sgx_init_test.obj
 0001:000021b8       WinMain                    000131b8 f   wince_unittests.obj
 0001:000023e0       ReleasePowerRequirement    000133e0 f   coredll:COREDLL.dll
 0001:000023f0       NKDbgPrintfW               000133f0 f   coredll:COREDLL.dll
 0001:00002400       FormatMessageW             00013400 f   coredll:COREDLL.dll
 0001:00002410       GetLastError               00013410 f   coredll:COREDLL.dll
 0001:00002420       SetPowerRequirement        00013420 f   coredll:COREDLL.dll
 0001:00002430       WideCharToMultiByte        00013430 f   coredll:COREDLL.dll
 0001:00002440       SGXGetMiscInfo             00013440 f   srvclum:SRVCLUM.dll
 0001:00002450       PVRSRVDisconnect           00013450 f   srvclum:SRVCLUM.dll
 0001:00002460       SGXReleaseClientInfo       00013460 f   srvclum:SRVCLUM.dll
 0001:00002470       PVRSRVCloseDCDevice        00013470 f   srvclum:SRVCLUM.dll
 0001:00002480       PVRSRVDestroyDeviceMemContext 00013480 f   srvclum:SRVCLUM.dll
 0001:00002490       PVRSRVUnmapDeviceClassMemory 00013490 f   srvclum:SRVCLUM.dll
 0001:000024a0       PVRSRVMapDeviceClassMemory 000134a0 f   srvclum:SRVCLUM.dll
 0001:000024b0       PVRSRVGetDCSystemBuffer    000134b0 f   srvclum:SRVCLUM.dll
 0001:000024c0       PVRSRVEnumDCDims           000134c0 f   srvclum:SRVCLUM.dll
 0001:000024d0       PVRSRVEnumDCFormats        000134d0 f   srvclum:SRVCLUM.dll
 0001:000024e0       PVRSRVGetDCInfo            000134e0 f   srvclum:SRVCLUM.dll
 0001:000024f0       PVRSRVOpenDCDevice         000134f0 f   srvclum:SRVCLUM.dll
 0001:00002500       PVRSRVCreateDeviceMemContext 00013500 f   srvclum:SRVCLUM.dll
 0001:00002510       PVRSRVEnumerateDeviceClass 00013510 f   srvclum:SRVCLUM.dll
 0001:00002520       SGXGetClientInfo           00013520 f   srvclum:SRVCLUM.dll
 0001:00002530       PVRSRVAcquireDeviceData    00013530 f   srvclum:SRVCLUM.dll
 0001:00002540       PVRSRVEnumerateDevices     00013540 f   srvclum:SRVCLUM.dll
 0001:00002550       PVRSRVConnect              00013550 f   srvclum:SRVCLUM.dll
 0001:000025e0       WinMainCRTStartup          000135e0 f   corelib0:pegwmain.obj
 0001:000026dc       exit                       000136dc f   corelib0:cexit.obj
 0001:000026f4       _exit                      000136f4 f   corelib0:cexit.obj
 0001:00002734       __GSHandlerCheckCommon     00013734 f   corelib0:gshandler.obj
 0001:00002770       __GSHandlerCheck           00013770 f   corelib0:gshandler.obj
 0001:00002794       __security_init_cookie     00013794 f   corelib0:seccinit.obj
 0001:000027f0       __security_check_cookie    000137f0 f   corelib0:armsecgs.obj
 0001:00002804       __gsfailure                00013804 f   corelib0:armsecgs.obj
 0001:00002848       _initterm                  00013848 f   corelib0:crt0dat.obj
 0001:0000287c       _cinit                     0001387c f   corelib0:crt0dat.obj
 0001:000028b0       printf                     000138b0 f   corelib1:COREDLL.dll
 0001:000028c0       sprintf                    000138c0 f   corelib1:COREDLL.dll
 0001:000028d0       strcmp                     000138d0 f   corelib1:COREDLL.dll
 0001:000028e0       free                       000138e0 f   corelib1:COREDLL.dll
 0001:000028f0       malloc                     000138f0 f   corelib1:COREDLL.dll
 0001:00002900       atol                       00013900 f   corelib1:COREDLL.dll
 0001:00002910       _stricmp                   00013910 f   corelib1:COREDLL.dll
 0001:00002920       _isctype                   00013920 f   corelib1:COREDLL.dll
 0001:00002930       wcslen                     00013930 f   corelib1:COREDLL.dll
 0001:00002940       memset                     00013940 f   corelib1:COREDLL.dll
 0001:00002950       _XcptFilter                00013950 f   corelib1:COREDLL.dll
 0001:00002960       __C_specific_handler       00013960 f   corelib1:COREDLL.dll
 0001:00002970       __security_gen_cookie2     00013970 f   corelib1:COREDLL.dll
 0001:00002980       __report_gsfailure         00013980 f   corelib1:COREDLL.dll
 0001:00002990       TerminateProcess           00013990 f   coredll:COREDLL.dll
 0001:000029bc       __IMPORT_DESCRIPTOR_COREDLL 000139bc     coredll:COREDLL.dll
 0001:000029d0       __IMPORT_DESCRIPTOR_SRVCLUM 000139d0     srvclum:SRVCLUM.dll
 0001:000029e4       __NULL_IMPORT_DESCRIPTOR   000139e4     coredll:COREDLL.dll
 0002:00000000       __imp_ReleasePowerRequirement 00014000     coredll:COREDLL.dll
 0002:00000004       __imp_NKDbgPrintfW         00014004     coredll:COREDLL.dll
 0002:00000008       __imp_FormatMessageW       00014008     coredll:COREDLL.dll
 0002:0000000c       __imp_GetLastError         0001400c     coredll:COREDLL.dll
 0002:00000010       __imp_SetPowerRequirement  00014010     coredll:COREDLL.dll
 0002:00000014       __imp_WideCharToMultiByte  00014014     coredll:COREDLL.dll
 0002:00000018       __imp___report_gsfailure   00014018     corelib1:COREDLL.dll
 0002:0000001c       __imp___security_gen_cookie2 0001401c     corelib1:COREDLL.dll
 0002:00000020       __imp___C_specific_handler 00014020     corelib1:COREDLL.dll
 0002:00000024       __imp__XcptFilter          00014024     corelib1:COREDLL.dll
 0002:00000028       __imp_memset               00014028     corelib1:COREDLL.dll
 0002:0000002c       __imp_wcslen               0001402c     corelib1:COREDLL.dll
 0002:00000030       __imp__isctype             00014030     corelib1:COREDLL.dll
 0002:00000034       __imp__stricmp             00014034     corelib1:COREDLL.dll
 0002:00000038       __imp_atol                 00014038     corelib1:COREDLL.dll
 0002:0000003c       __imp_malloc               0001403c     corelib1:COREDLL.dll
 0002:00000040       __imp_free                 00014040     corelib1:COREDLL.dll
 0002:00000044       __imp_strcmp               00014044     corelib1:COREDLL.dll
 0002:00000048       __imp_TerminateProcess     00014048     coredll:COREDLL.dll
 0002:0000004c       __imp_sprintf              0001404c     corelib1:COREDLL.dll
 0002:00000050       __imp_printf               00014050     corelib1:COREDLL.dll
 0002:00000054       \177COREDLL_NULL_THUNK_DATA 00014054     coredll:COREDLL.dll
 0002:00000058       __imp_PVRSRVConnect        00014058     srvclum:SRVCLUM.dll
 0002:0000005c       __imp_PVRSRVEnumerateDevices 0001405c     srvclum:SRVCLUM.dll
 0002:00000060       __imp_PVRSRVAcquireDeviceData 00014060     srvclum:SRVCLUM.dll
 0002:00000064       __imp_PVRSRVEnumerateDeviceClass 00014064     srvclum:SRVCLUM.dll
 0002:00000068       __imp_PVRSRVCreateDeviceMemContext 00014068     srvclum:SRVCLUM.dll
 0002:0000006c       __imp_PVRSRVOpenDCDevice   0001406c     srvclum:SRVCLUM.dll
 0002:00000070       __imp_PVRSRVGetDCInfo      00014070     srvclum:SRVCLUM.dll
 0002:00000074       __imp_PVRSRVEnumDCFormats  00014074     srvclum:SRVCLUM.dll
 0002:00000078       __imp_PVRSRVEnumDCDims     00014078     srvclum:SRVCLUM.dll
 0002:0000007c       __imp_PVRSRVGetDCSystemBuffer 0001407c     srvclum:SRVCLUM.dll
 0002:00000080       __imp_PVRSRVMapDeviceClassMemory 00014080     srvclum:SRVCLUM.dll
 0002:00000084       __imp_PVRSRVUnmapDeviceClassMemory 00014084     srvclum:SRVCLUM.dll
 0002:00000088       __imp_PVRSRVDestroyDeviceMemContext 00014088     srvclum:SRVCLUM.dll
 0002:0000008c       __imp_PVRSRVCloseDCDevice  0001408c     srvclum:SRVCLUM.dll
 0002:00000090       __imp_SGXReleaseClientInfo 00014090     srvclum:SRVCLUM.dll
 0002:00000094       __imp_PVRSRVDisconnect     00014094     srvclum:SRVCLUM.dll
 0002:00000098       __imp_SGXGetMiscInfo       00014098     srvclum:SRVCLUM.dll
 0002:0000009c       __imp_SGXGetClientInfo     0001409c     srvclum:SRVCLUM.dll
 0002:000000a0       \177SRVCLUM_NULL_THUNK_DATA 000140a0     srvclum:SRVCLUM.dll
 0002:000000a4       __security_cookie          000140a4     corelib0:seccinit.obj
 0002:000000a8       __security_cookie_complement 000140a8     corelib0:seccinit.obj
 0002:000000ac       pfnRegisteredWndProc       000140ac     wince_unittests.obj
 0002:000000b0       _exitflag                  000140b0     corelib0:cexit.obj
 0002:000000b4       __onexitend                000140b4     <common>
 0002:000000b8       __onexitbegin              000140b8     <common>

 entry point at        0001:000025e0

 Static symbols

 0001:000010cc       GetString                  000120cc f   sgx_init_test.obj
 0001:000012e8       SGXUT_query_sgx_corerev    000122e8 f   sgx_init_test.obj
 0001:00002568       WinMainCRTStartupHelper    00013568 f   corelib0:pegwmain.obj
 0001:00002614       doexit                     00013614 f   corelib0:cexit.obj
